:1000000000308A003D280000000000002D308400F0
:100010000008031919280130A100A001A00B0E2827
:10002000A10B0D284830A000A00B14280000800B65
:100030000B280034BE1B2D280F30A0003D0EA0055C
:100040000A302002031827283030A00729283E084C
:10005000A00720080C1E2A2899000F30BD050A3081
:100060003D020318352830303728BE133E08BD073F
:100070003D080C1E392899000034840183019F300B
:100080008400073080000C308316990026309800D9
:10009000903083129800A601A5019F308400803023
:1000A00080001F083839C1389F000030A1001F08A8
:1000B000C73921049F000130AD0006201F151F190C
:1000C0005F281E08A30083161E088312A7002308BA
:1000D000A8000830A1001F08C73921049F00013083
:1000E000AD0006201F151F1973281E08A3008316D4
:1000F0001E088312A9002308AA002030A1001F08AF
:10010000C73921049F000130AD0006201F151F19BB
:1001100087281E08A30083161E088312AB0023083D
:10012000AC002608AD00AE0126080039B000250855
:10013000AF002808B100B20128080039B400270830
:10014000B3002A08B500B6012A080039B80029080A
:10015000B7002C08B900BA012C080039BC002B08E4
:10016000BB002D08BD005730BE001A202F08BD006F
:100170005730BE001A203108BD00D730BE001A200B
:100180003308BD005730BE001A203508BD00D730F7
:10019000BE001A203708BD005730BE001A203908AB
:1001A000BD00D730BE001A203B08BD005730BE004E
:1001B0001A200A300C1EDA289900A50A0319A60A8B
:0401C000552863005B
:02400E00F23F7F
:00000001FF
